:020000040000FA
:020000000528D1
:06000A008312850183163C
:10001000FB30850061308F001A309F00D2308100A4
:1000200083128312073099000D309F000511851946
:10003000172805159F149F181B289F111E08A10043
:100040003D20A2000B11220881009F149F18262832
:100050009F151E08A1004921A3005522A4001030BD
:10006000900023088F0024088E000C1010140B1D24
:10007000372805110C1C3A2817282108A000493000
:10008000A00700300318013E8A002008482008001D
:1000900082000C340D340D340E340F34103410340F
:1000A0001134123412341334143415341534163414
:1000B00017341834183419341A341B341B341C34D4
:1000C0001D341D341E341F34203420342134223496
:1000D0002334233424342534253426342734283457
:1000E000283429342A342B342B342C342D342E3418
:1000F0002E342F34303430343134323433343334DA
:100100003434353436343634373438343934393499
:100110003A343B343B343C343D343E343E343F345B
:10012000403441344134423443344434443445341B
:100130004634463447344834493449344A344B34DD
:100140004C344C344D344E344F344F34503451349D
:10015000513452345334543454345534563457345F
:1001600057345834593459345A345B345C345C3421
:100170005D345E345F345F346034613462346234E1
:1001800063346434643465346634673467346834A3
:1001900069346A346A346B346C346D346D346E3463
:1001A0006F346F3470347134723472347334743425
:1001B00075347534763477347834783479347A34E5
:1001C0007A347B347C347D347D347E347F348034A7
:1001D0008034813482348334833484348534853468
:1001E000863487348834883489348A348B348B3429
:1001F0008C348D348D348E348F34903490349134EB
:1002000092349334933494349534963496349734AA
:100210009834983499349A349B349B349C349D346C
:100220009E349E349F34A034A134A134A234A3342C
:10023000A334A434A534A634A634A734A834A934EE
:10024000A934AA34AB34AC34AC34AD34AE34AE34AF
:10025000AF34B034B134B134B234B334B434B43470
:10026000B534B634B734B734B834B934B934BA3431
:10027000BB34BC34BC34BD34BE34BF34BF34C034F2
:10028000C134C134C234C334C434C434C534C634B4
:10029000C7342108A0005530A00701300318013EE3
:1002A0008A0020085421080082003C3456346A3405
:1002B0007A34863491349A34A134A834AD34B234CB
:1002C000B734BB34BE34C134C434C734C934CC347D
:1002D000CE34D034D134D334D434D634D734D834E3
:1002E000DA34DB34DC34DD34DE34DF34DF34E03484
:1002F000E134E234E234E334E434E434E534E53444
:10030000E634E634E734E734E834E834E934E93411
:10031000E934EA34EA34EB34EB34EB34EC34EC34E7
:10032000EC34ED34ED34ED34ED34EE34EE34EE34C3
:10033000EE34EF34EF34EF34EF34EF34F034F034A4
:10034000F034F034F034F134F134F134F134F13488
:10035000F134F234F234F234F234F234F234F2346E
:10036000F334F334F334F334F334F334F334F43454
:10037000F434F434F434F434F434F434F434F4343D
:10038000F434F534F534F534F534F534F534F53426
:10039000F534F534F534F534F634F634F634F63411
:1003A000F634F634F634F634F634F634F634F634FD
:1003B000F634F734F734F734F734F734F734F734E6
:1003C000F734F734F734F734F734F734F734F734D5
:1003D000F734F734F834F834F834F834F834F834BF
:1003E000F834F834F834F834F834F834F834F834AD
:1003F000F834F834F834F834F834F834F834F9349C
:10040000F934F934F934F934F934F934F934F93484
:10041000F934F934F934F934F934F934F934F93474
:10042000F934F934F934F934F934F934F934F93464
:10043000F934F934F934FA34FA34FA34FA34FA344F
:10044000FA34FA34FA34FA34FA34FA34FA34FA343C
:10045000FA34FA34FA34FA34FA34FA34FA34FA342C
:10046000FA34FA34FA34FA34FA34FA34FA34FA341C
:10047000FA34FA34FA34FA34FA34FA34FA34FA340C
:10048000FA34FA34FB34FB34FB34FB34FB34FB34F6
:10049000FB34FB34FB34FB34FB34FB34FB34FB34E4
:1004A000FB34FB34FB34FB34FB342108A000613007
:1004B000A00702300318013E8A00200860220800CD
:1004C0008200F534C73492343934E93468343B342B
:1004D000C0343E34E634DF3447343534BD34ED3493
:1004E000D1347434DD3414341E340234C2346334F1
:1004F000E8345334A734E63413342D3438343534E7
:1005000024340634DD34AA346D342634D7348034B0
:100510002234BD345134DF346734EA346834E13492
:100520005634C63432349B34FF346134BF341A3409
:100530007234C7341A346A34B73402344B349234C8
:10054000D7341A345B349A34D83413344E34863466
:10055000BE34F33428345B348D34BE34ED341C3473
:1005600049347634A134CB34F5341D3445346B34FE
:100570009134B634DB34FE3421344334653485346D
:10058000A534C534E434023420343D345A3476344E
:100590009134AD34C734E134FB3414342D34453454
:1005A0005D3475348C34A334B934CF34E534FA3443
:1005B0000F34243438344C346034733486349934F2
:1005C000AC34BE34D034E234F3340434153426343D
:1005D0003734473457346734763486349534A4340A
:1005E000B334C134D034DE34EC34FA340734153447
:1005F00022342F343C344934563462346E347B34E4
:10060000873493349E34AA34B534C134CC34D734CF
:10061000E234ED34F83402340D34173421342B3401
:1006200035343F34493453345C3466346F34783471
:1006300082348B3494349D34A534AE34B734BF3413
:10064000C834D034D834E134E934F134F9340134E5
:100650000834103418341F3427342E3436343D34E3
:1006600044344B3452345934603467346E34753406
:100670007C34823489348F3496349C34A334A93446
:10068000AF34B634BC34C234C834CE34D434DA34A3
:10069000DF34E534EB34F134F634FC340134073420
:1006A0000C34123417341D34223427342C343234B1
:1006B00037343C34413446344B3450345534593457
:0206C0005E34A6
:02400E00C430BC
:00000001FF
